:020000020000FC
:1000000019C094C01895ECC0DDC01895D7C01895DC
:10001000FCC000C118951895189518951895189555
:10002000ECC01895189542423133205374617274B4
:10003000204F4B3704E00EBF0FE50DBF01E00FBBB3
:100040000FEF0EBBE09A0DB301BF00E008BB00E06C
:1000500007BB00E005BB0AE204BB00E002BB08E30B
:1000600001BB02E003BF02E00EBD77278827992776
:1000700090937600909377009093BF009093240123
:10008000BB27A0E600270D93A438E8F39460FF2473
:10009000CED302E3B02EB4D1AE9A79D294FDFDCF87
:1000A0000CE002E192FD08E4302E06EF202E00273E
:1000B000C02ED02E009381000093820005E108BF7E
:1000C00009BF0FEF02BF002705BD002705BD04BD16
:1000D000106408B7012B08BF09B7006409BF789402
:1000E00003E005BF00E40BBF2AE083FFFECF092D2C
:1000F0001A2D877F0C541440B8F72A95B1F7F8945D
:1001000046D245D2AE9893FD42D27894F9E07F7DF5
:10011000706167D280D335D3379800B7086000BFCD
:1001200000917700046000937700C5C41FB6442790
:100130004BBF45B740FF1EC0829B3CC042E045BF5D
:100140004CB55DB5742E852E9F7B60917300461B68
:1001500060917400560B483A61E6560730F448390E
:100160006AE3560710F0906425C0BB2018F587FF9E
:10017000BA9420C082991EC043E045BF83FD1AC0D7
:100180004CB55DB5409373005093740096FF12C058
:100190009F7B47195809942EA52E483968E05607C9
:1001A00020F7403263E0560700F388604B2D42335E
:1001B00008F4B39450E45BBF1FBE18951FB67E7F52
:1001C0001FBE18951FB6442775FDAD9874FDA998FC
:1001D00074FD03C075FD01C0959845BD1FBE1895FF
:1001E0001FB642B343FD04C0939A949AAB9A03C0DE
:1001F00093989498AB981FBE18951FB645B34F7D42
:1002000045BB4427642E1FBE18951FB643948068D3
:100210001FBE18951FB676FD8BC0422D562D541764
:1002200088F43A94C1F452E192FD58E4662D641BBF
:10023000603328F06695669566956695560F352E5F
:100240004A9508C041F03A9431F458E092FD52E4E6
:10025000352E4395242E706474FF20C081FFAB9827
:1002600080FD1BC000000000000000000000000036
:10027000000000000000000000000000000000007E
:10028000000000000000000000000000000000006E
:1002900000000000000081FFA99A41C075FF20C046
:1002A00081FF939880FD1BC000000000000000004B
:1002B000000000000000000000000000000000003E
:1002C000000000000000000000000000000000002E
:1002D0000000000000000000000081FFAD9A1FC078
:1002E00081FF949880FD1BC000000000000000000A
:1002F00000000000000000000000000000000000FE
:1003000000000000000000000000000000000000ED
:100310000000000000000000000081FF959A422DBF
:100320004C59409542BF479544BD41E045BD64C02E
:10033000422D42BF7F7B74FF1AC0A99800000000C5
:1003400000000000000000000000000000000000AD
:10035000000000000000000000000000000000009D
:10036000000000000000000080FFAB9A39C075FF5C
:100370001CC0AD980000000000000000000000005C
:10038000000000000000000000000000000000006D
:10039000000000000000000000000000000000005D
:1003A0000000000080FF939A1BC095980000000099
:1003B000000000000000000000000000000000003D
:1003C000000000000000000000000000000000002D
:1003D00000000000000000000000000080FF949A70
:1003E0004C3918F482608E7F07C0463F18F08D7F2D
:1003F000816002C08D7F8E7F91FD81601FBE189548
:10040000F89400279860C19A0000000000000000E6
:100410000000B1999860B19B977FC19800B7077FA2
:1004200000BF06E007B9002741E055E0076006B9C4
:10043000379AC1D0FF24369A3699FECF04B115B150
:10044000369AF39415E0F116B9F7FF24369A3699E7
:10045000FECF04B115B1FF2039F4FF24F3941093BB
:100460006A0000936B00F2CF30916A0020916B001C
:10047000201B310B90F34427552730916A002091BF
:100480006B00020F131F451F469517950795109394
:100490006A0000936B00F39415E0F116B9F6FF249F
:1004A00037980027076006B90027066407B900914E
:1004B0006B0010916A00FF2493FD03C022E330E03B
:1004C00002C024E830E0F394021B130BE0F7FA9427
:1004D00093FD03C010E002E302C010E008E9222708
:1004E00033274F2D200F311F4A95E1F700916B0004
:1004F00010916A00201B310B08F4F394F092700005
:1005000093FD05C010E000E250E045E104C010E0BA
:1005100008E650E049E522273327200F311FFA94DF
:10052000E1F720936C0030936D0022273327F09081
:100530007000240F351FFA94E1F720936F00309379
:100540006E0005EC10E020916C0030916D003117C9
:1005500020F400936C0010936D000027056006B92D
:100560003798FF2400B7086000BF23EB30E093FD0D
:1005700004C020916F0030916E0000916B001091CB
:100580006A00021B130B08F008959460089510E8A8
:10059000002702BFAD9A949A02B70032E9F7AD98EE
:1005A000949828E0002702BF02B70F3FE9F72A9589
:1005B000C9F71A9569F710E828E0002702BF02B7CB
:1005C0000F3FE9F72A95C9F71A95B1F7089530E07A
:1005D0003BBF30E03EBD32E00CB51DB5242D3EBD25
:1005E0000895F5DF30E43BBF009360001093610095
:1005F00020936200C0916300D0916400E091650097
:100600000C1B1D0B2E0B34E02695179507953A957C
:10061000D9F7C02FD12FE22F2223A9F41093720013
:10062000112329F0EE240852134268F40EC0EE2084
:1006300011F41FEFE12E122D159515951A5C011777
:1006400020F4C12F02C0E7D032C0C0936600D0931F
:10065000670092FD1EC0022D00950535D0F00C2FCD
:100660001D2F1695079516950795169507951695BE
:1006700007953327262D209533952695E9F73A954A
:10068000532E22273327200F311F5A94E1F7C20F30
:10069000D31F92FD08C0D695C7950C2F1D2F169518
:1006A0000795C00FD11FC0936800D09369000091D7
:1006B000600010916100209162000093630010932C
:1006C000640020936500089583FF02C002D08DD09E
:1006D000089583FF24C0092D1A2D877F0C541440E0
:1006E00010F400271127169507951695079516956E
:1006F0000795202F0456104008F024E692FF0EC004
:100700002A3060F02F2F2A3018F411272AE0210F09
:10071000F39406E90F1510F02395FF24F22F0895A6
:1007200087FF18C08F7772FF06C07B7F4C2D453046
:1007300098F4C39403C0CC2009F0CA9471FF07C099
:100740007D7FAE984D2D443628F4D39403C0DD2030
:1007500009F0DA944AD008956AD0F8946BCC7160AD
:10076000C0916600D091670032DFC00FD11F05E451
:1007700009BFDBBDCABD05E509BF30E43BBF70FD65
:10078000FECF379800B7086000BF716020DFC0EB74
:10079000D6E30C0F1D1F25E429BF1BBD0ABD25E5AF
:1007A00029BF30E43BBF0895716011DFC09168003C
:1007B000D09169000C0F1D1F25E429BF1BBD0ABD88
:1007C00025E529BF30E43BBF82FD0BDF84FD81DFDF
:1007D00085FDA6DF77FD7AD286FD5AD292FF02C050
:1007E00097FD089570FDFECF08950F2F0D1908F4A1
:1007F00009E010917200183028F012E3011740F060
:10080000012F06C0143020F014E6011708F0012F64
:100810000095602E089506EF202E08E000937200E8
:10082000C8E2D3E2C0936600D0936700089506EF54
:10083000602E00E093989498AB98AD989598A998FD
:1008400002E1302E81609D7F8D7F9460089504E0E9
:100850000A95F1F7089590FD2DC0E9DF10E5002716
:1008600005BD04BD0FEF10917500011B03BD00E431
:1008700005BD08B710681F7B08BF09B70F7B0F774E
:1008800009BF05B5026005BD939A949AAB9A87FF9C
:10089000FECF8F771F931DDF1F91FD3008F00AC038
:1008A00003B520917500021B08F4002703BD1A95BB
:1008B00071F79160002705BD04BD08B710641F776C
:1008C00008BF09B700640F7709BFB1DF08959B7FA8
:1008D00070FD03C0F9DED39408C04599F8CFB7DFA7
:1008E0004599F5CF706860DF7F779598000000002C
:1008F0000000000080FFAD9A02E007B930DF70FD14
:1009000002C0D39408C0459BFACFA1DF459BF7CF27
:1009100080614ADF8F7E04E509BF7F7D7F7E81FD98
:1009200002C076FD03C0AB9880FF949A05E509BF2D
:1009300000E007B914DF70FD02C0D39406C04599EA
:10094000FACF85DF4599F7CF2FDFAD980000000083
:100950000000000080FFA99A04E007B900DF70FDE5
:1009600002C0D39408C0459BFACF71DF459BF7CFF7
:1009700080641ADF8F7B04E509BF70627F7E81FD92
:1009800002C076FD03C0949880FF939A05E509BFE5
:1009900002E007B9E4DE70FD03C0D394C1DE08C0F5
:1009A0004599F9CF54DF4599F6CF8062FDDE8F7D02
:1009B000A998000000000000000080FF959A00E068
:1009C00007B9CDDE70FD02C0D39408C0459BFACFB5
:1009D0003EDF459BF7CF8460E7DE8B7F04E509BFF0
:1009E0007F7D706181FD02C076FD03C0939880FF1A
:1009F000AB9A05E509BF04E007B9B1DEBB2061F0A1
:100A000091FD08C080FF06C026DF9E7F946002E350
:100A1000B02E51C09B7F5BCFF8940CCB777F002723
:100A20001127222730E104E007B900270000000069
:100A300045990160102F2A9549F0459911600000F1
:100A4000459B1E7F1017B9F3786008953A9599F782
:100A500008959498AB9893989598A998AD9873FD3C
:100A6000089594FD08959061F894A99A00000000FB
:100A7000939A949A002711270000000000000000BC
:100A80000395D1F70000000000009498002711277B
:100A9000000000000395E1F700000000A998949879
:100AA000939800000000000000000000000000001B
:100AB00000007894089508DE946090689F7E0FEFA0
:100AC000E02EDD24ABDF1AEF73FD1FEFE12E04E013
:100AD00007B9009182000093810073FD06C00027D2
:100AE0000093810080FDE7CF00C070FD02C09062DE
:100AF00006C04599FACFABDE4599F7CF55DE9598FC
:100B00000000000080FFAD9A02E007B99D7F0E2D26
:100B10000D3F29F00C3F19F00B3F09F001C0926026
:100B20001EDE0E2D083C08F49F7770FD02C0906217
:100B300008C0459BFACF8BDE459BF7CF806134DE42
:100B40008F7E04E509BF7F7D7F7E81FD02C076FD3B
:100B500003C0AB9880FF949A05E509BF00E007B990
:100B6000FEDD70FD02C0906206C04599FACF6FDECF
:100B70004599F7CF19DEAD980000000080FFA99AD3
:100B800004E007B9ECDD70FD07C090620E2D04365D
:100B900009F4449899DD06C0459BF5CF58DE459B86
:100BA000F2CF02DE04E509BF70627F7E81FD02C0E4
:100BB00076FD03C0949880FF939A05E509BF02E093
:100BC00007B99D7F0E2D013051F0EA940E2D0430AF
:100BD00029F0033019F0023009F001C09260BFDD46
:100BE00070FD02C0906208C04599FACF30DE459989
:100BF000F7CF8062D9DD8F7DA9980000000080FFCB
:100C0000959A00E007B90E2D18EC73FD16E901174F
:100C100008F49B7FA4DD70FD08C0906273FD03C0E3
:100C20000E2D043B08F4DDDC08C0459BF4CF0FDE3D
:100C3000459BF1CF8460B8DD8B7F04E509BF7F7DE4
:100C4000706181FD02C076FD03C0939880FFAB9A6E
:100C500005E509BF04E007B982DD91FD02C080FD12
:100C60002ACF0091760095FD00270395009376002A
:100C700095FDD3949F7D023018F4BB2041F034CF12
:100C80009B7F9F77EE2420DD02E003BF20CEC4CE01
:100C900086FF089507B10093710007E007B900B718
:100CA000077F00BF379A00000000369A3699FECFC2
:100CB0008F7B04B115B1043108F07460209171008C
:100CC00027B9379820B7286020BF089577FF089587
:100CD00007B10093710006E007B900B7077F00BFB6
:100CE000379A00000000369A3699FECF04B115B14C
:100CF0007F772091710027B9379820B7286020BFEF
:100D000020916C0030916D00201B310B80F07260DF
:100D1000AE9A8D7F23EB30E093FF04C020916F00EB
:100D200030916E00201B310B10F005E0D00EFF2437
:100D30000895A895F8941FBB0EBBE09AE099FECFEA
:100D40000DB378940895A895F894E199FCCF0EBB63
:0C0D50001FBB2DBBE29AE19A7894089535
:00000001FF
